:10000000B601052AB80071218413FA30A600A701B1
:10001000EA21A00AA50AA201A30100083805A6004A
:10002000640000083805A7002606270538060319CE
:10003000A20A0319A30A2708A600A4030319A5030B
:100040000319A00B10282208002AB616B61EB612F5
:10005000B6192E28B6156920031855280830A300B4
:100060007E20A20DA30B3028B61E6020882084209D
:10007000B61A55205A2022080310002AB616B61EBA
:10008000B61236194828FE39B70036150310002A73
:10009000361A5028A6003616692003185528260857
:1000A000712003185528B61E002A602088203611BA
:1000B0003612B6113A08840038088417800466287E
:1000C0003A08840038098005841780056728682865
:1000D000002A5A2088200422602084203708B6197C
:1000E0000138A2000830A300A20D03185A20031CF7
:1000F000602088208420A30B74285A2088203A0886
:10010000840038080005FF3E3B0884003909632855
:100110003B08840039085D28A400B7172730A300E6
:1001200010309E200330A300E8309E20A3016430ED
:100130009E20A3010A309E202408A928A200250899
:10014000A1002408A000CE212008031DB713B71B6F
:100150000800303EA700071187108710831607118B
:1001600087108710F030860583122708B618D62826
:100170003A30A1009830AC213330A600EB20133088
:10018000A1008830AC21EB206430AB21EB2064303F
:10019000AB212230A600EB202830D5200C30D52012
:1001A0000630D520B6142708D6283614A600361CEB
:1001B000E4288710033C031CE928E9200730A1004C
:1001C000D030AC21031408003614FE3C0319002A79
:1001D0008714A60E361C36100715F0308605260843
:1001E0000F3986040711A60E3618EB283230AB21E2
:1001F00003140800B800841780048413A201201C93
:10020000A20008210319002A08210319002A08293D
:100210003808A2060130A000A10100083805220616
:10022000031D0800A00A0319A10F0D290800A5014C
:10023000A400B7172730A30010302A210330A300F1
:10024000E8302A21A30164302A21A3010A302A219F
:1002500024083529A2002508A1002408A000CE21E9
:100260002008031DB713B71B0800303EA6003A084C
:1002700084000930A70003104221A60CA70B3C29DB
:10028000031442298413B71D512900083804371D6F
:1002900038068000841700083804031C38068000E4
:1002A0005C2900083804031C38063719380680001A
:1002B0008417380980055C29370D0639A0006521AF
:1002C000A100A00A65210000AC2901308A002008A5
:1002D00082070134993403343934003460340C34E7
:1002E000FD3484178004002AA000A00DA00DA00DED
:1002F0003830A005813020049F000030A10032304A
:10030000AC211F151F1982291E08A1001E08002AF2
:1003100003178D0083168C130C1483120C08002A0B
:1003200003178C0083168C130C1555308D00AA30E2
:100330008D008C148C189A290C11002AA301A2009C
:10034000FF30A207031CA307031C002A0330A100EF
:10035000E730AC21A029A101FC3EA000A109031CAB
:10036000B729FF300000A0070318B229A0076400D6
:10037000A10FB1290800A2000130BE29A80023085E
:100380002102031DC5292208200204300318013070
:10039000031902302805031DFF30002A1030A60083
:1003A000A501A401210DA40DA50D2208A402230876
:1003B000031C230FA5020318E4292208A40723081D
:1003C0000318230FA5070310A00DA10DA60BD2291A
:1003D0002008002A1030A800A101A001A70CA60C3B
:1003E000031CF8292208A00723080318230FA107DC
:1003F000A10CA00CA50CA40CA80BEE292408002A23
:10040000831303138312640008008316EF30850002
:1004100004309F00703086008113870183128501AC
:1004200086018701071083160710643083129E210E
:100430008A11DB2AFE30AA200130AA204830AA20E7
:100440006530AA206C30AA206C30AA206F30AA2018
:100450002030AA202130AA202130AA200330A30076
:10046000E8309F21FE30AA200130AA205930AA206E
:100470004130AA205430AA204130AA204930AA2075
:100480002330AA203230AA202030AA205430AA20BB
:100490004530AA205330AA205430AA202030AA2068
:1004A0005030AA205230AA204F30AA204730AA202C
:1004B0005230AA204130AA204D30AA200130A3009A
:1004C000F4309F21FE30AA20C030AA20B130AA20EB
:1004D000B530AA202030AA20B730AA20B030AA20F8
:1004E0002030AA207430AA206F30AA202030AA2001
:1004F0005330AA207430AA206130AA207230AA207A
:100500007430AA206400061B822A08000130A00073
:10051000053084000430FA202008CE002108CF00E6
:100520000800E830A2000330A30005308400043046
:100530000220CC002308CD00080000307421D00038
:1005400014309E21080001307421D10014309E2106
:1005500008000730BA001030B8000730BB00083080
:10056000B900A030402045084020440840205008F1
:100570004020510840204F0840204E083E200A30BD
:100580009E2108000730BA001030B8000730BB00C9
:100590000830B900A03040204508402044084020E1
:1005A0002720D0002720D1002720CF002520CE00F3
:1005B0000A309E2108001A22FE30AA200130AA200B
:1005C000B130AA20B530AA203A30AA204C30AA2057
:1005D0006F30AA206730AA202030AA20B730AA2086
:1005E0002030AA203A30AA205030AA206C30AA200D
:1005F0006130AA207930AA20FE30AA20C030AA207B
:10060000B130AA20B630AA203A30AA205330AA200E
:100610007430AA206F30AA207030AA202030AA207F
:100620004C30AA206F30AA206730AA200130A300E6
:10063000F4309F2164008A11061F252B8A11640063
:100640008A11861E762C8A111A2BC401C501440812
:10065000A0004508A1001F30A3004030BB218A1133
:10066000031D1F2C8A114408A0004508A100043076
:10067000A200A301CE21C8002108C9009D22A32207
:10068000862203104E0DC6004F0DC7000730BA007A
:100690004030B8000230B700443036216130362196
:1006A0007430362161303621233036213D303621F9
:1006B0002C3036214908A500480818212C30362155
:1006C0002030362141303621303036213D30362140
:1006D0002C3036213F08A5003E0818212E30362147
:1006E0003D08A5003C0818212C3036212030362149
:1006F00041303621313036213D3036212C30362103
:100700004308A500420818212E3036214108A500D3
:10071000400818212C303621203036214330362134
:1007200048303621323036213D3036212C303621CA
:100730004708A500460818210D3036210A30362119
:100740005008A000A1010A30A200A301CE21BE00E2
:100750002108BF005008A000A1010A30A200A30197
:10076000CE212408BC002508BD005108A000A1012D
:100770000A30A200A301CE21C2002108C300510803
:10078000A000A1010A30A200A301CE212408C000CC
:100790002508C100FE30AA200130AA204430AA203A
:1007A0002330AA203D30AA204908A50048088C2003
:1007B0002030AA204330AA204830AA203230AA2074
:1007C0003D30AA204708A50046088C20FE30AA200C
:1007D000C030AA204130AA203030AA203D30AA20C3
:1007E0003F08A5003E088C202E30AA203D08A50019
:1007F0003C088C205630AA202030AA204130AA2064
:100800003130AA203D30AA204308A50042088C20A0
:100810002E30AA204108A50040088C205630AA207E
:10082000A92232309E2164008A11061E202C8A11D2
:100830000430C407031C272BC50A031D272BDC2A01
:100840000130A300F4309F214408D3004408A000E5
:100850004508A100A2010130A300CE21D200031758
:1008600005308D00031353089021031706308D00C7
:10087000031352089021FE30AA200130AA205330E1
:10088000AA207430AA206F30AA207030AA204C30E1
:10089000AA206F30AA206730AA206730AA206930CA
:1008A000AA206E30AA206730AA20FE30AA20C030CD
:1008B000AA204530AA204E30AA204430AA20203059
:1008C000AA204430AA206130AA207430AA206130C6
:1008D000AA202330AA203D30AA204908A5004808B4
:1008E0008C201330A30088309F21DC2AFE30AA2000
:1008F0000130AA20B130AA20B530AA203A30AA206F
:100900005030AA206C30AA206130AA207930AA2069
:100910002030AA20B730AA202030AA203A30AA20BE
:100920005330AA207430AA206530AA207030AA2043
:10093000FE30AA20C030AA20B130AA20B630AA20AA
:100940003A30AA204530AA204E30AA204430AA20AE
:100950000330A300E8309F2164008A11061FBA2CDF
:100960008A1164008A11861E0C2E8A116400061EEC
:10097000DC2AAC2C05308821D30006308821D20037
:100980005208A600A701A2010130A300EA21B2008B
:100990002508B30053083207CA0033080318013E84
:1009A000CB00C401C5014408A0004508A1004B08C4
:1009B000A3004A08BB218A11031DC82D8A114408CF
:1009C000A0004508A1000430A200A301CE21C80068
:1009D0002108C900C2225008A000A1010A30A200CB
:1009E000A301CE21BE002108BF005008A000A10134
:1009F0000A30A200A301CE212408BC002508BD00B6
:100A00005108A000A1010A30A200A301CE21C2001A
:100A10002108C3005108A000A1010A30A200A301CF
:100A2000CE212408C0002508C10003104E0DC600C9
:100A30004F0DC700FE30AA200130AA204430AA2062
:100A40002330AA203D30AA204908A50048088C2060
:100A50002030AA204330AA204830AA203230AA20D1
:100A60003D30AA204708A50046088C20FE30AA2069
:100A7000C030AA204130AA203030AA203D30AA2020
:100A80003F08A5003E088C202E30AA203D08A50076
:100A90003C088C205630AA202030AA204130AA20C1
:100AA0003130AA203D30AA204308A50042088C20FE
:100AB0002E30AA204108A50040088C205630AA20DC
:100AC00005309E210730BA004030B8000230B70030
:100AD0004430362161303621743036216130362180
:100AE000233036213D3036212C3036214908A500EF
:100AF000480818212C30362120303621413036214B
:100B0000303036213D3036212C3036213F08A500CB
:100B10003E0818212E3036213D08A5003C0818213A
:100B20002C303621203036214130362131303621EB
:100B30003D3036212C3036214308A50042081821CB
:100B40002E3036214108A500400818212C303621CE
:100B5000203036214330362148303621323036219C
:100B60003D3036212C3036214708A5004608182193
:100B70000D3036210A30362164008A11061ECD2D33
:100B80008A110430C407031CD32CC50A031DD32CBF
:100B90001330A30088309F21DC2AFE30AA200130C8
:100BA000AA205330AA207430AA206F30AA207030B7
:100BB000AA202030AA205030AA206C30AA20613010
:100BC000AA207930AA206230AA206130AA2063309E
:100BD000AA206B30AA20FE30AA20C030AA204530BF
:100BE000AA204E30AA204430AA202030AA20443027
:100BF000AA206130AA207430AA206130AA202330B4
:100C0000AA203D30AA204908A50048088C200B30B6
:100C1000A300B8309F21DC2A05308821D30006309C
:100C20008821D2005208A600A701A2010130A3002A
:100C3000EA21B2002508B30053083207CA0033087E
:100C40000318013ECB00C401C5014408A0004508BB
:100C5000A1004B08A3004A08BB218A11031D1F2FC6
:100C60008A114408A0004508A1000430A200A30195
:100C7000CE21C8002108C900C2220730BA00403086
:100C8000B8000230B700443036216130362174306C
:100C9000362161303621233036213D3036212C304B
:100CA00036214908A500480818212C30362120306B
:100CB000362141303621303036213D3036212C303E
:100CC00036213F08A5003E0818212E3036213D0868
:100CD000A5003C0818212C30362120303621413027
:100CE0003621313036213D3036212C303621430833
:100CF000A500420818212E3036214108A5004008E1
:100D000018212C303621203036214330362148300E
:100D10003621323036213D3036212C3036214708FD
:100D2000A500460818210D3036210A30362150081A
:100D3000A000A1010A30A200A301CE21BE0021081B
:100D4000BF005008A000A1010A30A200A301CE21DB
:100D50002408BC002508BD005108A000A1010A30EC
:100D6000A200A301CE21C2002108C3005108A000A7
:100D7000A1010A30A200A301CE212408C000250849
:100D8000C10003104E0DC6004F0DC700FE30AA2053
:100D90000130AA204430AA202330AA203D30AA20C6
:100DA0004908A50048088C202030AA204330AA20FA
:100DB0004830AA203230AA203D30AA204708A5009A
:100DC00046088C20FE30AA20C030AA204130AA203C
:100DD0003030AA203D30AA203F08A5003E088C20D4
:100DE0002E30AA203D08A5003C088C205630AA20B1
:100DF0002030AA204130AA203130AA203D30AA203C
:100E00004308A50042088C202E30AA204108A500E6
:100E100040088C205630AA2055309E2164008A114B
:100E2000061E242F8A116400061B0E2F64309E219B
:100E30000430C407031C252EC50A031D252E1330BC
:100E4000A30088309F21DC2AFE30AA200130AA208E
:100E50005330AA207430AA206F30AA207030AA2004
:100E60002030AA205030AA206C30AA206130AA205D
:100E70007930AA206230AA206130AA206330AA20EB
:100E80006B30AA20FE30AA20C030AA204530AA200C
:100E90004E30AA204430AA202030AA204430AA2074
:100EA0006130AA207430AA206130AA202330AA2001
:100EB0003D30AA204908A50048088C200B30A3002B
:0A0EC000B8309F21DC2A6300632F85
:02400E00763DFD
:00000001FF
